:100000001CC0D5C173C132C00AC230C02FC02EC0BF
:100010002DC02CC02BC02AC029C028C027C026C094
:1000200025C024C023C0ABC0B8C0BBC0C5C0CFC0B2
:10003000D6C0DFC0E7C0EEC0FDC011241FBECFEDAB
:10004000CDBF10E0A0E6B0E0E8EDF4E002C005901E
:100050000D92A236B107D9F710E0A2E6B0E001C0D8
:100060001D92AC36B107E1F71CD134C2C9CF889AD2
:100070009098D09AD8988C9A9498899A91988D9AB9
:100080009598BC9AC498BE9AC698BF9AC798D19AB8
:10009000D998BA9AC298BD9AC598B898C09A8E9ABB
:1000A0009698909AD89A949A919A959AC49AC69A40
:1000B000C79AD99AC29AC59A08951092630010926D
:1000C000620009C080916200909163000196909354
:1000D000630080936200809162009091630021E050
:1000E000843F920778F308951092630010926200A3
:1000F00009C0809162009091630001969093630023
:1001000080936200809162009091630023E0883EBA
:10011000920778F308951092670090E002C0845629
:10012000922F292F2F5F8436D0F7909366009091FD
:10013000670002C08A50922F292F2F5F8A30D0F794
:10014000909367008093680080916600882319F47B
:100150008AE080936600809166008A3031F4909145
:100160006700992311F4809367000895E82FF0E069
:10017000EA30F10508F06BC0ED5EFF4F09949198ED
:100180009598C498C698C798D99897DF919A959AE8
:10019000C49AC69AC79AD99A08959598C4988DDF3B
:1001A00036C091989598C698C798C29886DF919A5C
:1001B000959AC69AC79A3CC091989598C498C69843
:1001C000C2987BDF919A959AC49AC69A31C0959845
:1001D000C498D998C29871DF959AC49A28C091980A
:1001E000C498C698D998C29868DF919AC49AC69A5A
:1001F0001EC09198C498C698C798D998C2985DDFD8
:10020000919A12C091989598C49857DF919A959AAF
:10021000C49A089591989598C498C698C798D99803
:10022000C2984BDF919A959AC49AC69AC79AD99A5E
:10023000C29A089591989598C498C698D998C298EA
:100240003CDF919A959AC49AC69AD99AC29A08950F
:100250009098809166008ADF909A46DFD8988091C6
:10026000670084DFD89A40DF9498809168007EDF31
:10027000949A3ADF08958FE085BF80EC8BBF089594
:1002800084E690E09BBD8ABD1FBC8EB588608EBDA4
:100290001DBC1CBC8EB581608EBD89B7806489BFD2
:1002A00008950F931F93CF93DF937894E4DFDFDEFD
:1002B000E7DFCAE0D0E080916100813069F480918D
:1002C000600029DF00E010E0C3DF0F5F1F4F083C34
:1002D0001105D1F710926100809164009091650042
:1002E000BE01E4D0862F17DFB3DFE5CF1F920F9258
:1002F0000FB60F9211242F938F939F9380916000DC
:100300008230E1F0833020F4813009F048C006C02B
:10031000833029F1843009F042C034C080916400F8
:1003200090916500B09906C025E08C3D9207B8F524
:1003300001962CC0009799F1019728C08091640024
:1003400090916500B09906C025E0823D9207E0F4E7
:100350000A961CC08B309105F0F00A9717C0809167
:10036000640090916500B09907C025E08837920736
:1003700058F48C599F4F0AC08536910560F0845619
:10038000904004C0B09907C08CED95E09093650053
:100390008093640004C010926500109264009F91E5
:1003A0008F912F910F900FBE0F901F9018951F9255
:1003B0000F920FB60F9211242F933F934F935F9399
:1003C0006F937F938F939F93AF93BF93EF93FF931D
:1003D000F8948ADE89DE88DE87DE86DE7894809176
:1003E00060008F5F8093600080916000853018F01E
:1003F00081E08093600081E080936100FF91EF9144
:10040000BF91AF919F918F917F916F915F914F912C
:100410003F912F910F900FBE0F901F9018951F9234
:100420000F920FB60F9211242F933F938F939F93A8
:1004300080916A0090916B00009749F4969A8091A0
:10044000640090916500805E9C4F9BBD8ABD809149
:100450006A0090916B008130910559F4969880E480
:1004600091E52091640030916500821B930B9BBD48
:100470008ABD80916A0090916B00019690936B0009
:1004800080936A0080916A0090916B0082309105A0
:1004900021F410926B0010926A009F918F913F910E
:1004A0002F910F900FBE0F901F901895AA1BBB1B8A
:1004B00051E107C0AA1FBB1FA617B70710F0A61B64
:1004C000B70B881F991F5A95A9F780959095BC0185
:0804D000CD010895F894FFCF5F
:0204D800010120
:00000001FF
